:1000000015C0189518951895189518951895189560
:100010001895A5C9189518951895189518951895B7
:100020001895189518951895189518958FE181BD14
:1000300087E181BD8FE58DBFC0E4E8E34E2E82E00D
:100040008EBFD2E0F2E05F2EEEEFF1E0A0E6B0E08E
:1000500088278D933197E9F78AE189B988E18AB9D0
:1000600056DA662483E086B9379A85E083BF8D9A95
:100070008C9A81EA8FBD80E08EBD8FEF81BB8FEFC0
:1000800087BB82E08EBD89B7816089BF789480E0AC
:100090008093C20080E090E0AEEBB0E08D939C9343
:1000A00080E08093610080E08093600088EC90E0C5
:1000B000A4EBB0E08D939C938CE390E0A6EBB0E0D2
:1000C0008D939C938CE291E0AAEBB0E08D939C938E
:1000D0008CE291E0ACEBB0E08D939C9383E0809355
:1000E000CB0085E08093CC008CE291E0A5ECB0E001
:1000F0008D939C938CE291E0A7ECB0E08D939C9360
:1001000082E08093CD0080E090E09BBD8ABD80E0DE
:1001100090E099BD88BDF0D98CE045DAE8E0F0E0E8
:10012000A2EDB0E091E02BDB0091D2000B3709F09B
:1001300041C0EAE0F0E0ACEBB0E092E020DBECE0C4
:10014000F0E0A4EBB0E092E01ADBEEE0F0E0A6EB2A
:10015000B0E092E014DBE0E1F0E0AAEBB0E092E086
:100160000EDBE2E1F0E0ABECB0E091E008DBE4E1D3
:10017000F0E0ACECB0E091E002DB0091CC000230AA
:1001800008F003C082E08093CC004091CB00009146
:10019000CC00041708F004C08091CB008093CC0001
:1001A0000091CC00093010F009F001C003C089E0D3
:1001B0008093CC0004D50091D0000A3009F001C032
:1001C000DAD500916100003009F03DC0F8D400910B
:1001D000D000093009F037C0929A81E08093610025
:1001E00081E080936000A2E6B0E0ECE8F7E16DD931
:1001F00088D9A2E6B0E078D988EE93E027DAA2E6C3
:10020000B0E0E2EAF7E161D9ABE8B0E0ECEBF0E0B6
:100210004BDAABE8B0E05FD9E8EBF7E156D9ABE8F1
:10022000B0E059D9E4EBF0E03FDAABE8B0E053D905
:10023000E0ECF7E14AD965D9A2E6B0E055D95AD940
:10024000ABE8B0E051D900916100013009F0AFC1D5
:10025000B6D40091D000003108F0A9C10091D000BF
:10026000093009F012C080E08093610080E0809343
:100270006000A2E6B0E0E8ECF7E127D9ABE8B0E037
:10028000E8ECF7E122D938D992980091D0000730F4
:1002900009F00FC0A0E6B0E08C918F5F8C930091C5
:1002A0006000043010F009F001C003C082E08093C8
:1002B00060000091D000053009F00DC0A0E6B0E06C
:1002C0008C9181508C9300916000023008F003C043
:1002D00084E0809360000091D000063009F003C0F4
:1002E00081E08093600000916000013009F041C01E
:1002F0000091D0000B3009F03CC082E08093610097
:1003000080E080936000A2E6B0E0EEEDF7E1DDD89A
:10031000ABE8B0E0E8ECF7E1D8D88091C200809378
:10032000C40080E08093CE00969AAAEBB0E00D91D5
:100330001C914BE050E07DD8A4EDB0E04D935C9370
:10034000A4EDB0E00D911C914FEF50E00423152374
:10035000A4EDB0E00D931C93A4EDB0E08D919C91C1
:1003600099BD88BD85E087B980D9A4EDB0E08D93B3
:100370009C930091D0000A3009F058C000916000B1
:10038000023009F01DC0ACEBB0E00D911C9141E0D2
:1003900050E0040F151FACEBB0E00D931C93ACEBD9
:1003A000B0E00D911C91083552E0150714F009F0EA
:1003B00001C006C088E592E0ACEBB0E08D939C9361
:1003C00000916000033009F01DC0A4EBB0E00D9176
:1003D0001C9141E050E0040F151FA4EBB0E00D9319
:1003E0001C93A4EBB0E00D911C91043F51E0150764
:1003F00014F009F001C006C084EF91E0A4EBB0E076
:100400008D939C9300916000043009F00FC0ADEC17
:10041000B0E08C918F5F8C930091CD00033010F091
:1004200009F001C003C083E08093CD000091D000AB
:10043000013009F054C000916000023009F01CC086
:10044000ACEBB0E00D911C9141E050E0041B150BAA
:10045000ACEBB0E00D931C93ACEBB0E00D911C91B4
:10046000013050E015070CF401C006C081E090E0B7
:10047000ACEBB0E08D939C9300916000033009F0E9
:100480001CC0A4EBB0E00D911C9141E050E0041BB6
:10049000150BA4EBB0E00D931C93A4EBB0E00D9111
:1004A0001C91013050E015070CF401C006C081E03A
:1004B00090E0A4EBB0E08D939C9300916000043039
:1004C00009F00DC0ADECB0E08C9181508C9300919F
:1004D000CD00013008F003C081E08093CD00009191
:1004E0006000013009F01CC0A2E6B0E0E4EFF7E1E3
:1004F000ECD7ABE8B0E0ECEBF0E0D6D8ABE8B0E09E
:10050000EAD7EAE0F8E1E1D7ABE8B0E0E4D7E4EB22
:10051000F0E0CAD8ABE8B0E0DED7E2E1F8E1D5D749
:1005200000916000023009F010C0A2E6B0E0EAE1FC
:10053000F8E1CBD7ABE8B0E0ECEBF0E0B5D8ABE856
:10054000B0E0C9D7E0E3F8E1C0D700916000033024
:1005500009F010C0A2E6B0E0E2E4F8E1B6D7ABE8FB
:10056000B0E0E4EBF0E0A0D8ABE8B0E0B4D7E8E569
:10057000F8E1ABD700916000043009F010C0A2E6AA
:10058000B0E0EAE6F8E1A1D7ABE8B0E0EDECF0E0EE
:1005900092D8ABE8B0E09FD7E2E8F8E196D7B1D7C0
:1005A000A2E6B0E0A1D7A6D7ABE8B0E09DD7009116
:1005B0006100023009F093C002D30091D0000031F5
:1005C00008F01BC00091D0000B3009F00EC081E094
:1005D00080936100A2E6B0E0E4E9F8E176D7ABE809
:1005E000B0E0E8ECF7E171D778D68BD7A2E6B0E0BF
:1005F0007BD780D7ABE8B0E077D74091C2000091BD
:10060000C400041709F46BC08091C2008093C40039
:1006100051D2ABE8B0E0EAEAF8E157D7ABE8B0E096
:100620005AD7E8EBF0E040D8ABE8B0E054D7E2EBC3
:10063000F8E14BD78FEDABE8B0E08F934CD78F91BB
:100640008D9388278C93ABE8B0E045D7E4EBF8E1D5
:100650003CD750D7ABE8B0E047D7A6EBB0E04D9120
:100660005C91A8EBB0E00D911C91041715070CF0FC
:1006700001C035C083E080936100A2E6B0E0ECEBFE
:10068000F8E123D781EEA2E6B0E08F9324D78F91D3
:100690008D9388278C93A2E6B0E01DD7E6ECF8E1B5
:1006A00014D72FD7A2E6B0E01FD780E090E0AEEBE2
:1006B000B0E08D939C9380E08093C20080E08093B3
:1006C000C900A4EBB0E00D911C9142E050E0D7D6F8
:1006D000BB27A4E18D919C919BBD8ABD979A009107
:1006E0006100033009F066C16AD20091D000003188
:1006F00008F01BC00091D0000B3009F00EC085E05F
:1007000080936100A2E6B0E0E4E9F8E1DED6ABE870
:10071000B0E0E8ECF7E1D9D6E0D5F3D6A2E6B0E058
:10072000E3D6E8D6ABE8B0E0DFD60091D0000630E3
:1007300009F004C080E08093C900C1984091C200D4
:100740000091C400041709F435C18091C200809360
:10075000C400B0D1ACEBB0E00D911C91AEEBB0E0B9
:100760004D915C91041B150BA0ECB0E00D931C9314
:100770000091CA00003009F032C0ABE8B0E0EEEC06
:10078000F8E1A3D6ABE8B0E0A6D6E0ECF0E08CD779
:10079000ABE8B0E0A0D6E8EBF7E197D6ABD6ABE894
:1007A000B0E0A2D6A2E6B0E0ECEBF8E18ED681EEA6
:1007B000A2E6B0E08F938FD68F918D9388278C938C
:1007C000A2E6B0E088D6E8EDF8E17FD69AD60091AF
:1007D000C900003009F003C0A2E6B0E085D6009160
:1007E000CA00023009F034C0ABE8B0E0EAEEF8E14C
:1007F0006CD6ABE8B0E06FD6E4EBF0E055D7ABE8F1
:10080000B0E069D6E8E5F8E160D674D6ABE8B0E0D0
:100810006BD684E087B929D7A4EDB0E08D939C9383
:10082000A4EDB0E00D911C91043F51E0150714F0C8
:1008300009F001C00DC0A2E6B0E0E2EFF8E145D654
:1008400060D6A2E6B0E050D6C19A81E08093C9009C
:100850000091CA00043009F053C0ABE8B0E0E8E012
:10086000F9E133D6ABE8B0E036D6E8EBF0E01CD7E0
:10087000ABE8B0E030D6E2EBF8E127D68FEDABE89D
:10088000B0E08F9328D68F918D9388278C93ABE817
:10089000B0E021D6EEE0F9E118D62CD6ABE8B0E016
:1008A00023D6A6EBB0E00D911C91A8EBB0E04D91E2
:1008B0005C91041B150BA4EDB0E00D931C93A4ED0B
:1008C000B0E08D919C91D5D5A4EDB0E08D939C9333
:1008D000A4EDB0E00D911C91043050E0150714F028
:1008E00009F001C00DC0A2E6B0E0ECE1F9E1EDD500
:1008F00008D6A2E6B0E0F8D5C19A81E08093C9009D
:100900000091CA00063009F023C0ACEBB0E00D91B5
:100910001C91AEEBB0E04D915C91041B150BA0EC6B
:10092000B0E00D931C93ABE8B0E0E2E3F9E1CDD584
:10093000ABE8B0E0D0D5EAEBF0E0B6D6ABE8B0E09B
:10094000CAD5EAE3F9E1C1D5D5D5ABE8B0E0CCD55D
:10095000AAECB0E08C918F5F8C930091CA000830B4
:1009600009F003C080E08093CA00A0ECB0E00D91D4
:100970001C91013050E015070CF401C01BC081E050
:1009800080936100A2E6B0E0E4E4F9E19ED5B9D538
:100990000091C900003009F003C0A2E6B0E0A4D580
:1009A000ABE8B0E0EAE5F9E190D5A4D5ABE8B0E07A
:1009B0009BD593D400916100053009F07AC0FFD037
:1009C0000091D000003108F057C00091D0000B30EA
:1009D00009F04AC083E080936100A2E6B0E0ECEB4E
:1009E000F8E173D581EEA2E6B0E08F9374D58F91D4
:1009F0008D9388278C93A2E6B0E06DD5E0E7F9E10E
:100A000064D57FD5A2E6B0E06FD5A4EBB0E00D9140
:100A10001C9142E050E033D5BB27A4E18D919C911D
:100A20009BBD8ABD979A969AAAEBB0E00D911C9156
:100A30004BE050E0FED4A4EDB0E04D935C93A4ED08
:100A4000B0E00D911C914FEF50E004231523A4ED6D
:100A5000B0E00D931C93A4EDB0E08D919C9199BDF5
:100A600088BD80E08093C9004CD5A2E6B0E03CD5BB
:100A700041D5ABE8B0E038D50091D000063009F0A0
:100A800018C081E08093610081E080936000A2E65D
:100A9000B0E0ECE7F9E119D534D5A2E6B0E024D511
:100AA000ABE8B0E0EAE5F9E110D524D5ABE8B0E079
:100AB0001BD587CB80E087B9D8D5A8EBB0E08D9364
:100AC0009C93A8EBB0E00D911C914EE150E0ACD4AA
:100AD000A8EBB0E00D931C93A8EBB0E00D911C9136
:100AE00043E351E0A6D4A8EBB0E04D935C93A8EBB0
:100AF000B0E00D911C914AE050E0040F151FA8EBE7
:100B0000B0E00D931C93A6EBB0E00D911C91A8EB07
:100B1000B0E04D915C91041B150BA4EDB0E00D937A
:100B20001C93A4EDB0E00D911C910F3050E015071F
:100B30000CF401C00EC00091CB004091CD00040F19
:100B4000AFECB0E00C93AFECB0E08C9182508C93A2
:100B50000DC00091CC004091CD00040FAFECB0E08F
:100B60000C93AFECB0E08C9182508C930091CE004E
:100B7000003009F00EC0A6EBB0E04D915C91A8EBFF
:100B8000B0E00D911C91041715070CF401C001C0D1
:100B9000939A4091CF000091CE00041709F001C054
:100BA0009398AEECB0E08C918F5F8C930091CE0067
:100BB000053109F003C080E08093CE000895809154
:100BC000D0008093D2000091D2000A3009F025C0F5
:100BD00080E18093D200A5ECB0E08D919C9136D558
:100BE000A5ECB0E00D911C9142E350E0041B150B05
:100BF000A5ECB0E00D931C93A5ECB0E00D911C9119
:100C0000023350E015070CF401C006C08AE090E002
:100C1000A5ECB0E08D939C9306C08CE291E0A5EC2E
:100C2000B0E08D939C930091D200013009F025C073
:100C300080E18093D200A7ECB0E08D919C9106D525
:100C4000A7ECB0E00D911C9142E350E0041B150BA2
:100C5000A7ECB0E00D931C93A7ECB0E00D911C91B4
:100C6000023350E015070CF401C006C08AE090E0A2
:100C7000A7ECB0E08D939C9306C08CE291E0A7ECCA
:100C8000B0E08D939C93B8D4A3EDB0E00C930091A9
:100C9000D300003109F419C0A3EDB0E08C918F703E
:100CA0008C934091D3000091D200041709F00DC03D
:100CB000A3D4A3EDB0E00C93A3EDB0E08C918F70C2
:100CC0008C9384E690E0C2D4ECCF96D4A0EDB0E053
:100CD0000C938AE090E0BAD48FD4402F0091D000DA
:100CE000041709F044C00091D000003109F43EC05F
:100CF000A0EDB0E08C918F708C930091610000307A
:100D000010F009F001C032C080E08093D200009161
:100D1000D200043610F009F029C0C09A80E0809318
:100D2000D3000091D300063210F009F007C0A3ED04
:100D3000B0E08C918F5F8C9309F0F3CFC09880E086
:100D40008093D3000091D300063210F009F007C061
:100D5000A3EDB0E08C918F5F8C9309F0F3CFA2EDFF
:100D6000B0E08C918F5F8C9309F0D1CF03C080E10C
:100D70008093D00008958AE080936100929A81E088
:100D800080936000A2E6B0E0E2E9F9E19ED3ABE82F
:100D9000B0E0E2E8F8E199D3B4D3A2E6B0E0A4D39E
:100DA000A9D3ABE8B0E0A0D30ADF0091D0000031B6
:100DB00008F059C20091D000073009F00DC0A0E63C
:100DC000B0E08C918F5F8C9300916000083009F047
:100DD00003C081E0809360000091D000053009F0ED
:100DE0000DC0A0E6B0E08C9181508C930091600022
:100DF000003009F003C088E0809360000091D000CB
:100E0000063009F027C081E08093610081E0809383
:100E10006000A2E6B0E0E4EAF9E157D3ABE8B0E065
:100E2000E6EBF9E152D3ABE8B0E0ECEBF0E03CD418
:100E3000ABE8B0E050D3E8EBF7E147D3ABE8B0E084
:100E40004AD3E4EBF0E030D4ABE8B0E044D3E0ECDC
:100E5000F7E13BD30091D0000A3009F0B0C0009117
:100E60006000023009F01DC0ACEBB0E00D911C91A8
:100E700041E050E0040F151FACEBB0E00D931C9364
:100E8000ACEBB0E00D911C91083552E0150714F061
:100E900009F001C006C088E592E0ACEBB0E08D93AC
:100EA0009C9300916000033009F01DC0A4EBB0E0FA
:100EB0000D911C9141E050E0040F151FA4EBB0E030
:100EC0000D931C93A4EBB0E00D911C91043F51E0F5
:100ED000150714F009F001C006C084EF91E0A4EBFF
:100EE000B0E08D939C9300916000043009F01DC028
:100EF000A6EBB0E00D911C9141E050E0040F151FEE
:100F0000A6EBB0E00D931C93A6EBB0E00D911C9105
:100F1000033650E0150714F009F001C006C083E65F
:100F200090E0A6EBB0E08D939C93009160000530BB
:100F300009F01DC0AAEBB0E00D911C914AE050E011
:100F4000040F151FAAEBB0E00D931C93AAEBB0E0C1
:100F50000D911C9108325AE0150714F009F001C0F8
:100F600006C088E29AE0AAEBB0E08D939C930091D2
:100F70006000063009F00FC0ABECB0E08C918F5FE1
:100F80008C930091CB00093010F009F001C003C030
:100F900089E08093CB0000916000073009F00FC01A
:100FA000ACECB0E08C918F5F8C930091CC00093059
:100FB00010F009F001C003C089E08093CC000091DB
:100FC000D000013009F0ABC000916000023009F0A0
:100FD0001CC0ACEBB0E00D911C9141E050E0041B53
:100FE000150BACEBB0E00D931C93ACEBB0E00D91A6
:100FF0001C91013050E015070CF401C006C081E0DF
:1010000090E0ACEBB0E08D939C93009160000330D6
:1010100009F01CC0A4EBB0E00D911C9141E050E040
:10102000041B150BA4EBB0E00D931C93A4EBB0E0F4
:101030000D911C91013050E015070CF401C006C061
:1010400081E090E0A4EBB0E08D939C930091600070
:10105000043009F01CC0A6EBB0E00D911C9141E0FA
:1010600050E0041B150BA6EBB0E00D931C93A6EB10
:10107000B0E00D911C91043150E015070CF401C053
:1010800006C084E190E0A6EBB0E08D939C930091C4
:101090006000053009F01CC0AAEBB0E00D911C9176
:1010A0004AE050E0041B150BAAEBB0E00D931C9333
:1010B000AAEBB0E00D911C910A3050E015070CF43A
:1010C00001C006C08AE090E0AAEBB0E08D939C934B
:1010D00000916000063009F00DC0ABECB0E08C91DF
:1010E00081508C930091CB00023008F003C082E065
:1010F0008093CB0000916000073009F010C0ACEC89
:10110000B0E08C9181508C934091CB000091CC0049
:10111000041708F004C08091CB008093CC000091AC
:101120006000013009F00AC0A2E6B0E0E2E9F9E1AE
:10113000CCD1ABE8B0E0E2E8F8E1C7D100916000C3
:10114000023009F010C0A2E6B0E0E8ECF9E1BDD150
:10115000ABE8B0E0ECEBF0E0A7D2ABE8B0E0BBD19D
:10116000E8EDF9E1B2D100916000033009F010C060
:10117000A2E6B0E0E8EEF9E1A8D1ABE8B0E0E4EB3C
:10118000F0E092D2ABE8B0E0A6D1E8EFF9E19DD172
:1011900000916000043009F01FC0A2E6B0E0E8E072
:1011A000FAE193D1ABE8B0E0E6EBF0E07DD2ABE85A
:1011B000B0E091D1EAE1FAE188D18FEDABE8B0E09F
:1011C0008F9389D18F918D9388278C93ABE8B0E072
:1011D00082D1EEE1FAE179D100916000053009F0A9
:1011E00010C0A2E6B0E0E8E2FAE16FD1ABE8B0E00F
:1011F000EAEBF0E059D2ABE8B0E06DD1E8E3FAE118
:1012000064D100916000063009F010C0A2E6B0E0A1
:10121000E8E4FAE15AD1ABE8B0E0EBECF0E04BD215
:10122000ABE8B0E058D1ECE5FAE14FD100916000B5
:10123000073009F010C0A2E6B0E0EAE6FAE145D1D5
:10124000ABE8B0E0ECECF0E036D2ABE8B0E043D194
:10125000ECE5FAE13AD155D1A2E6B0E045D14AD168
:10126000ABE8B0E041D100916100013009F09CCDC4
:10127000EAE0F0E0ACEBB0E092E07BE76FD2ECE0CC
:10128000F0E0A4EBB0E092E07BE768D2EEE0F0E0C3
:10129000A6EBB0E092E07BE761D2E0E1F0E0AAEB00
:1012A000B0E092E07BE75AD2E2E1F0E0ABECB0E0F4
:1012B00091E07BE753D2E4E1F0E0ACECB0E091E008
:1012C0007BE74CD28BE78093D200E8E0F0E0A2ED20
:1012D000B0E091E07BE742D20895969880E090E0FC
:1012E00099BD88BD979880E090E09BBD8ABD93989A
:1012F000C198089581D1A0EDB0E00C930091D00089
:10130000003109F414C0A0EDB0E08C918F708C9383
:10131000F8D0A2E6B0E0E0EDF0E0CDD1A2E6B0E09A
:10132000DAD0E0E8FAE1D1D0A2E6B0E0DDD0E2CF59
:10133000929A45DC0091D000003109F40FC0E1D051
:10134000A2E6B0E0E0EDF0E0B6D1A2E6B0E0C3D0B6
:10135000E0E8FAE1BAD0A2E6B0E0C6D0E9CF0F9259
:101360001F922F923F924F925F927F928F929F9205
:10137000AF92BF920F931F932F933F934F935F931F
:101380006F937F938F939F93AF93BF93CF93DF938D
:10139000EF93FF938FB78F93A3ECB0E08C918F5FA7
:1013A0008C930091C3000F3010F009F001C01CC0F5
:1013B00080E08093C300A2ECB0E08C918F5F8C93AF
:1013C0000091C2000C3309F00FC080E08093C2008E
:1013D000AEEBB0E00D911C9141E050E0040F151F01
:1013E000AEEBB0E00D931C938F918FBFFF91EF9107
:1013F000DF91CF91BF91AF919F918F917F916F912D
:101400005F914F913F912F911F910F91BF90AF909E
:101410009F908F907F905F904F903F902F901F9064
:101420000F901895F894FFCF08D043D000FC10D04F
:10143000089503D024D001F8F9CF0024E89457FF91
:1014400002C009D0689400F80BD010F80124089568
:1014500002D009D00895509540954F5F5F4F089591
:10146000E89417FF0895009510950F5F1F4F68943B
:10147000089599231AF48095909501960895352F33
:10148000242FE894452B11F468940895512F402F90
:101490000027112780E1440F551F001F111F021B59
:1014A000130B416018F4020F131F4E7F8A9599F7B2
:1014B00008950F92049F202C312C419F300C509F97
:1014C000030C022D102D0F900895C8950D923196A2
:1014D0000020D9F708958F938D918823E9F711970C
:1014E0008F910895A8E2B2E08D91882311F055D034
:1014F000FBCF089580EC57C081E055D005D080E83F
:1015000052C080E850D0089583E099279FC08AEFA9
:1015100090E09CD0BF9ABE9ABD9ABC9ABA9ABB9AE8
:10152000C398EF93FF93E5E6F0E05DD0FF91EF9174
:10153000C298C798C698C59AC49AC29AEF93FF9367
:10154000E5E6F0E050D0FF91EF91C2987CD0C29ACE
:10155000EF93FF93E5E6F0E046D0FF91EF91C2985C
:1015600072D0C29AEF93FF93E5E6F0E03CD0FF9192
:10157000EF91C29868D0C498C29AEF93FF93E5E6C2
:10158000F0E031D0FF91EF91C2985DD088E20BD0AE
:101590008EE009D086E007D00895C39A829505D0E1
:1015A00004D051D00895C398F9CF859510F4C49A0A
:1015B00001C0C498859510F4C59A01C0C598859559
:1015C00010F4C69A01C0C698859510F4C79A01C058
:1015D000C798C29AEF93FF93E5E6F0E004D0FF913D
:1015E000EF91C29808953197F1F70895689462F8E1
:1015F0000895E89462F8089500E18FEF85BB8FE0CD
:1016000084BB80EF85BB8AE08A95F1F79C9B00E064
:101610009D9B04E09E9B08E09F9B0CE080EF84BBB9
:101620008FE085BB8AE08A95F1F78827989B80E058
:10163000999B81E09A9B82E09B9B83E0080F8AE064
:1016400090E004D0089581E090E000C0EF93FF9314
:10165000EE27E82BE92B31F0E9E1F4E03197F1F7DF
:101660000197D1F7FF91EF910895369A3699FECF01
:10167000369A3699FECF84B195B10895000F111FA7
:10168000221F331F089500951095209530950F5F08
:101690001F4F2F4F3F4F0895019110810EC00191B0
:1016A0001191219130810BC00191108117FF05C06C
:1016B0003FEF2FEF04C0008111272227332737FF88
:1016C00003C0E1DF8DE28D93CF93DF93CF92DF9262
:1016D000EF92AA24BB24CC24DD24EE2440E2CAE00D
:1016E000DD2755E093E38881890F87FD9F7083FD97
:1016F000907F891B89935A95A9F7C0DFAA1CBB1C50
:10170000CC1CDD1CEE1C4A9551F7E894EFE0FF2756
:1017100082910ED0EB30E0F71EF068948A2D0CD049
:1017200088278D93EF90DF90CF90DF91CF91089530
:10173000982F829501D0892F8F70805D26F080339D
:1017400009F4089568948D930895E199FECFEEBB56
:10175000FFBB3196089591E001C092E07B3751F4D0
:101760007FB7F894F2DF8D918DBBE29AE19A9A955A
:10177000C9F77FBF7727089591E001C092E0E5DFC8
:10178000E09A8DB38D939A95D1F70895536F66744F
:10179000776172652056312E303261202020202062
:1017A00020004265726569742020202020202020BE
:1017B0002020202020202000206D696E2020200085
:1017C000206D4120202020002020202020202020CB
:1017D0002020202020202020202020200000416EDA
:1017E0006865697A656E2020202020202020202036
:1017F000202000004265726569742020202020208E
:1018000020202020202020200000206D696E202034
:101810000000206D4120202000005A6569742020BE
:1018200020202020202020202020202020200000F8
:10183000206D696E202020202020202020202020C4
:1018400020005374726F6D20202020202020202043
:101850002020202020200000206D4120202020205A
:1018600020202020202020202000566F6C756D65E0
:101870006E2020202020202020202020202020201A
:101880000000202020202020202020202020202098
:1018900020202000556E7465726272656368756EF3
:1018A0006720202020202020000054656D70203DFE
:1018B000200020004320202020200000566F726767
:1018C000616E67206C0075667420202020005265D0
:1018D00073747A6569742000756674202020202056
:1018E000202020202020202000005374726F6D20C3
:1018F00000005374726F6D6665686C6572212020FC
:10190000202020202020000054656D7020004320FE
:1019100020202020202020202020200054656D70D1
:101920006572617475726665686C6572212020202D
:101930000000447265687A2E20002052504D20200D
:1019400020202000566F7267616E67206265656EA9
:10195000646574202020202000004F4B2020202090
:1019600020202020202020202020202020200000B7
:10197000756674202020202020202000566F72677A
:10198000616E67206162676562726F6368656E2071
:101990002000536572766963652020202020202076
:1019A00020202000426572656974202020202020BC
:1019B0002020202020002020202020202020202047
:1019C00020202020202000005A656974202020203B
:1019D0002020202020200000206D696E2020202063
:1019E00020202020202000005374726F6D202020C2
:1019F0002020202020200000206D412020202020B9
:101A00002020202020200000536F6C6C74656D70C6
:101A10006572617475722020000020200000432050
:101A20002020202020200000447265687A61686CC4
:101A300020202020202000002052504D2020202057
:101A400020202020202000004865697A6C65697399
:101A500074756E6720202020202000002020202088
:101A600020202020202020202000416E6865697AF7
:101A70006C65697374756E6720202020202000003B
:041A80002020200002
:00000001FF
